:10000000830100308A001F28F00003088301A70045
:100010000A08A8008A01831203138C1E10281128D5
:1000200016281A08A000A201A20AA3010313831232
:1000300028088A0027088300F00E700E090020307F
:10004000840027302A2083010A128A11302F0406E7
:100050008001840A0406031900342728831203133D
:10006000A900AA1B3C282A1B44282A088A00290820
:10007000A90A0319AA0A820083132A1883172908D8
:08008000A90A84000008080031
:100D7C00831603131815193099001812831298173B
:100D8C008316981683121816031383120800831205
:100D9C000313A400D12E83160313981CD62ED72E22
:100DAC00D12E831203132408990003138312080015
:100DBC0083120313A500043083120313A4005330D1
:100DCC0083120313A600EB2EEB2E83120313A60B38
:100DDC00F02EF12EEA2E83120313A40BF62EF72E0F
:100DEC00E52E83120313A50BFC2EFD2EE12E03130F
:100DFC008312080083120313A401192F8312031307
:100E0C0024082407A9002508AA0029080318AA0AFF
:100E1C000A128A112E200A128A110A128A11CD2660
:100E2C000A128A11A40A8312031324082407A900A6
:100E3C002508AA0029080318AA0A0A128A112E20CA
:100E4C000A128A110038031D2C2F2D2F042F031387
:100E5C00831208000A300A128A11DE260A128A113D
:100E6C000A128A11BE260A128A11063083169F00B6
:100E7C00EF309200871007110C3083129D000C305C
:100E8C00970083160911881008118811091006148F
:100E9C000814051189108312121583160612831279
:100EAC0088100811881506160B1383168C128B13D9
:100EBC00632F831203139B01950183120313081CE8
:100ECC00682F692F5F2F83120313981C6E2F6F2FBF
:100EDC00732F181209141816762F83120313091086
:100EEC00831203138C1E7B2F7C2F8D2F18197F2FB1
:100EFC00802F842F89141A08A0008D2F83120313BE
:100F0C001808A1001A08A1001A08A0008910831261
:100F1C000313061C922F932F982F831203139B01FC
:100F2C009501932FD72F5A30831203139B0009116D
:100F3C00051164309500F02F4B308312031395008C
:100F4C000911051164309B00F02F3230831203130A
:100F5C0095000911051164309B00F02F83120313C7
:100F6C0095010911051564309B00F02F4B3083124D
:100F7C0003139B000911051164309500F02F3230DA
:100F8C00831203139B000911051164309500F02F97
:100F9C00831203139B010915051164309500F02F82
:100FAC00F02F831203132008013A0319CE2F033AB2
:100FBC000319C52F063A0319BC2F0C3A0319992FA4
:100FCC00183A0319A22F303A0319AB2F603A0319C0
:100FDC00B42FF02F83120313103086062203230440
:100FEC00031DF92FFA2FFC2FA201A301692F0A125E
:040FFC008A111F280F
:02400E00393D3A
:00000001FF
